:020000021000EC
:1000000000C00091780005FD0AC1F092400608E1A9
:10001000009353060FEF0A950023E9F70091480675
:1000200003FFECC0E0E0F0E0079116910F3F19F4F8
:100030001F3F09F4E3C0F3C03BB72BBFF801209189
:10004000CA014093CA013DE930933400E8952093FA
:10005000CA013BBF08953091CF0137FDFCCF3BB7BC
:100060002BBFF8012091CA0113E21093CA010A01C3
:10007000E8952093CA013BBF089527E402EA10E007
:100080000E94FF800E94668178940E944F840E94A3
:100090008584FFCF009190290F770093C3040895C2
:1000A00000919029002319F0025039F005C024E096
:1000B00030E007E111E218C03CC020E004EE10E29D
:1000C00050E032E0F0E0E22FEC51FF4D42A1239FDF
:1000D000F801E00DF11D428353832395203190F305
:1000E00022E22093E42030E027D001E0089554D0AC
:1000F000018D0A9529F00A95A1F00A95B9F019C069
:10010000E0ECF0E2228930E0729615D045D0048D03
:10011000158D20A131A10217130710F400A311A31C
:10012000E4CFE0ECF0E222813381EFCFB9DF0023AE
:1001300069F700E008958F010C949E842DD0068904
:100140000F7109F0F6CF1789068907FF11C0112337
:1001500029F0165039F0125031F0F4CF22E030E09F
:10016000B69604C0C4CF21E030E0BC96E4DFBDCF3A
:10017000155019F0145031F0E5CF0AE410E802A34D
:1001800013A3F5CF01E010E006A317A3008D04A789
:10019000002369F30C949881E8E7F9E20895FCDF05
:1001A00000E000A301A302A303A304A305A30689FF
:1001B00007FF05C0048D158D012B09F4BACF0091FE
:1001C0008E29007621F4BADF002309F08ECF00914A
:1001D0008E290F71013091F70E94B4810023B1F78D
:0201E000EDCF61
:1001F4000C94A7840C94DF8407C040E04BBFF80143
:1002040058ED54BF2083089501E70DBF00E20EBFEF
:10021400C7E5DAE20E9427872EDFF09253060091A9
:100224000020109101200A3A154511F00C940000A9
:10023400F0920020F092012000E200937800F6CFC3
:100244004091CA01E22FF32F0093CA010491409315
:10025400CA010895BA01A801890102D199C261E0D5
:100264006A93BA01A901FCD0A7C2B90198018B0114
:1002740022C20E94F386D801C9012A0106C0FC01EA
:100284002191CF018D0129D2119682012FEF420EC7
:10029400521E012BA1F7E6E00C94FF8662E770E2A0
:1002A400260F371F0C940A876AE271E2F9CFF8949B
:1002B4000AEA15E5E0E0F0E2008311832091790079
:1002C400216009E731D0FFCF24E001E42DD02DE1F6
:1002D40027D0009362002CE123D0009363001FB762
:1002E400F894E0E5F0E00081026000831FBF009114
:1002F400510001FBE6F721E000E410E018D2E6E546
:10030400F0E00081097F008300E807870BEB008B96
:10031400008104600083E0E60081016000830895A9
:1003240030E002E00C94228110E001C200E000936E
:10033400342159D00091900000932A21009191001A
:1003440000932B210091920000932C2100919300A3
:1003540000932D210091D00101FB16F001E001C0B2
:1003640000E0D4C04FD4AEE8B9E200918E29007603
:100374000032B9F510918F290C91569707FF15C0DB
:10038400125049F01A9551F526E030E004E211E2EA
:1003940028D101E027C0BED00289138920E00030B3
:1003A4001207E1F0F80109951DC01A9521F01350C8
:1003B400A9F419D0EECF00913421002331F009E5DE
:1003C40011E892960D931C93E4CF20E430E007E308
:1003D40011E207D10FEF11E89496F4CF9BD00FE010
:1003E40073D000E00CC400C000E0B5D0ABD200E094
:1003F40004A305A302A303A30895F5DF10E08AD0A4
:10040400128B138BE7E3F1E230812181203001E08C
:10041400300709F428C0203003E0300709F43CC059
:100424002130300709F454C0203004E0300761F46F
:100434000091CF0107FDFCCF40E200E011D00E9403
:100444001C8097D100E062C02330300721F401E022
:100454000093342108952330364009F448C0ABC0DA
:1004640020E030E0089556D0018D128D012309F06B
:100474006FC0268137812030304011F424D002C06F
:100484001DD009F498C020E038E0A9D007E413E8AF
:1004940059D204A315A33CC011D019F021D011F4F2
:1004A40012D089C0018D128D012319F00AEA12E8D5
:1004B40002C00FED12E8028B138B2AC009E311E28C
:1004C40050D00023089503E000870AE004870895CC
:1004D400F5DF19F005D011F4F6DF6DC083D018C034
:1004E400ECE1F1E224813581203030400895E7E3E6
:1004F400F1E20281002349F40381013108F055C07F
:100504000CD000E007D0048B058B02C0009335218A
:1005140001E00895ECE1F1E20895033041F0023086
:1005240031F0043021F0053011F011E001C010E089
:100534001093362112E0019FF001E356FF4D6081D4
:10054400F1810CE111E2E62F48E050E00C94E386DF
:1005540003E001D030C00093242102E0009328215D
:100564000895BD01F80150810181402FA0E3B1E25B
:100574000D935C935597128130E0038120E00D9038
:100584001D902D903C9013970015110522053305FD
:1005940010F00BD008C0041B150B0F5F1F4FFD019B
:1005A400068B178B01E0DB01089508E000932421FA
:1005B4000AE00093282100E0089524D3ACE1B1E2DD
:1005C400FD014689578951D01496ED91FC911597F8
:1005D4000995FD012689378902D001E010C308E797
:1005E40011E2AAC190D0ACE1B1E2FD0106891789FC
:1005F400012B39F400E018EF068B178B80E098E0AC
:1006040010C0FD0106891789202F212B59F11830BC
:1006140010F4C80102C080E098E0081B190B068B97
:10062400178BAC0122D06481F581E62F099508E788
:1006340011E207C0FD01248935892F5F3F4F248BC8
:10064400358B9C010197232BE1F2F80121918F0155
:100654002F3F81F305E0009324210CE313E8FD010F
:10066400028B138BE4E00C9401872489358908E715
:1006740011E208954FDF248905890093782120939E
:10068400792122E030E0ABDF43CF44DF04891589D0
:1006940046895789202F2F73622F70E028E731E2B3
:1006A400260F371F6681F781E62F099500E04AD1AE
:1006B40004A305A32DCFB90132D0208127FDFDCF9E
:1006C400ECEC208128602083105F98018B01EADD27
:1006D400ECECF1E00081077F21CE15D0C801A22FF8
:1006E400B091CA0112D01BD0008107FDFDCF3AD0D2
:1006F4009093C1018093C001A093C40105E312D07B
:10070400B093CA01AFCF0C94F58609D0008107FDE0
:10071400FDCF008101FF02C006E304D00895EFEC91
:10072400F1E008950093CA0121E00BEC11E00C9470
:10073400FF809A938A93802F9091CA01E6DF0091FB
:10074400CF0107FDFCCF0ED00093C1010093C0017F
:100754008093C40103950032C8F39093CA01899130
:100764009991089503E30093CA0100E00093C20144
:1007740008958A930FEFDDDFD2DF008107FDFDCFFF
:100784008091CA0100E3CEDF8093CA018991089564
:100794002091CF0127FDFCCF262F272B61F0F801F4
:1007A40030E03BBF2691FA012193AF010F5F1F4F49
:1007B40061507040F1CF08950E94EE8622974A015D
:1007C4002B016D84D801912F80E007C04091CF01A7
:1007D40047FDFCCF45E20E941C80042D052909F445
:1007E40042C0AA240091CF0107FDFCCF00E8702E7F
:1007F400662071F0FC0130E03BBF0791169108833D
:10080400198308810F3F1F4F31F0AA24A39403C01A
:100814000FEF08830983042D052979F0A817B90778
:1008240029F425D00883042D052939F0FC013196DB
:10083400AE17BF0711F41BD00983488159818C017D
:100844000FDE0E942B8002967A9491F6AC015A95A1
:10085400AA208A0105DE09F0B9CF4091CF0147FDF6
:10086400FCCF44E2B8CF2296ECE00C94FA860FEF6A
:10087400400E501E1196F40101914F0108952AE192
:1008840007D00093FA042BE103D00093FB040895EE
:1008940047DD0F3F09F40FE108950E94F68600E05A
:1008A4000093600023E004E43FDD6DD20064008324
:1008B40001E0009360000FB7F894A02FD1DD890107
:1008C400E6D0F801E858F64D358323952230B8F385
:1008D400D6DF0091C0040093C00455D200680083A1
:1008E40000810061008388E799E20496E6EC808346
:1008F4009183E0EC32D10FEF0583E8EC0DDDAFBF5F
:10090400E3E00C9402871FB7F89400E439D200E2C4
:1009140037D2E1ECF4E000DDE9EC00810260008311
:10092400E8EC008100640083E9ECF6DCE8EC00818B
:10093400006800831FBF089505D0068F178F20A37A
:1009440031A30895E8E7F9E2089565D00091CB0456
:1009540007FF02C000E82EC0FCD1002361F5EBECD8
:1009640013D204FF1EC000E10BD200E00093A429BF
:1009740001E010E000939E2910939F2900E000936A
:10098400C30420E430E05AD020E430E010E000E872
:1009940055D007EA19E200938029109381292ED1BA
:1009A4000AC0008106FF02C000E404C0008105FF04
:1009B40002C000E2E5D11CD018952DD0E8D1002367
:1009C400B1F402E00093CC040091C50422D0F801F4
:1009D400008105FF06C01DD020E2F801269315D141
:1009E40006C000E817D020E2F8012693B9D0E3CF7F
:1009F4009BBF8FBF099119912991399149915991BF
:100A0400699179910990199029903990E991F99116
:100A1400A6CE00E02DC09A938A93FA93EA933A9271
:100A24002A921A920A927A936A935A934A933A931D
:100A34002A931A930A938FB79BB708958A932051E8
:100A4400304041F02051304039F02052304031F0F4
:100A540080E005C081E003C082E001C083E0DADF0A
:100A640020E0F801218326E02083806481838ECEF8
:100A74006CE779E2202F2F70220F402F440F00E003
:100A840010E0001F020F03D0060F171F089543E064
:100A94000C94DD869D01E8EC77D10F7D0083008105
:100AA4000F7D00833FD102E00593A6E8B9E200E0A0
:100AB40010E00D930C93539600E2069300E4069322
:100AC4003BD1069300E406931D931D931D931C9341
:100AD40015971D931C9311A7D90108950CD10023D8
:100AE40031F0033011F0043009F429D187D02ADF22
:100AF40006811781083050E0104039F548E027EAB4
:100B040039E20EE819E2CEDBE8ECF4E026D025D099
:100B14000E94CF80002309F4F1C014DF068907FF87
:100B24000BC000A10F7311F401E001C000E006A79F
:100B34000ED002E005A714C0048D158D012B09F415
:100B440005C005D001E005A7F3D00895E3C000E097
:100B540000A701A702A703A7089500810062DECBC6
:100B640051D0C7D0033011F448D046C0FD0120A1B4
:100B740031A142A553A58901041B150B402F412B1C
:100B840021F506A5002311F4D0D036C000A511A587
:100B9400020F131F248D358D0217130728F089D0F7
:100BA40019F00995002339F400E00093A629FD010A
:100BB400068707871FC070D020A111A1022F2F73B1
:100BC40011F421E001C020E026A7013420E012073F
:100BD40010F000E410E006871787268D378D42A5B4
:100BE40053A5240F351F208B318B9A01200F311F01
:100BF40022A733A797D09DD002C0A1D04BCFA991F3
:100C0400B9910895BA93AA9308957DDD72D0043002
:100C140011F4F3DF40C0FD018681978162A573A5BD
:100C240020A131A18B01080F191F2017310718F4D7
:100C3400C901861B970BAC0127EA39E2068D178D93
:100C4400060F171F2FDBFD0102A513A5080F191F9F
:100C540002A713A78034904031F426D0448D558DDB
:100C64002417350760F000A311A394966FD029F0E0
:100C74000995002311F442D00EC04CD00CC020A121
:100C840031A12017310731F414D0A9F309950023B9
:100C940091F302D04DD0E6CCFD0102A513A504D0FA
:100CA40020A731A700E056CF20A531A5200F311F82
:100CB40008959496ED91FC91959700E0E030F0074B
:100CC400089500917C2905FD07C015D0013009F471
:100CD4003DCF043009F415D008950091842905FD11
:100CE40007C009D0023009F420C0033009F409D048
:100CF4000895A8E7B9E20091A529089505E00093B5
:100D0400A529E5E8F9E204E00593EDE7F9E204E05A
:100D14000593089517DE03E005A700E0068707871B
:100D240001D007C0E4E8F9E2089504E00093A5299E
:100D340003D002E006930895ECE7F9E2089562DF38
:100D4400AAE9B9E203D009F0099559CFED91FC91D4
:100D5400B4CFEBEC19D002FF07C0F093CA040091A2
:100D6400842906FDAEDFD4CB008101FF08C002E078
:100D740007D000917C2906FFF6CFAFDFF4CF1BCC60
:100D84000093CA040895E0ECF4E000810895009112
:100D9400CC0400FF10CC01E00093CC04CDDF00E8CC
:100DA4000693C0DF00E8069301E0EADFC5DF00E157
:100DB400069394DEADCB4A951AF0000F111FFBCFBA
:100DC4000895AF93BF93D80101900D9241505040C4
:100DD400D9F7BF91AF910895AA929A928A927A9282
:100DE4006A925A924A92BA93AA939A938A930895CA
:100DF400AA84998488847F806E805D804C80BB81C6
:100E0400AA8199818881F0E0EC0FFD1FEF0108951C
:100E1400BD01D801F90104C021912D9341505040E6
:100E2400242F252BC9F7DB01089520E008D0E9F72A
:100E340008953BBF27913BB702D0D9F708952D936E
:100E440001501040202F212B08950EEA402E0EE071
:100E5400502E01E0602EF201362D6BBE07911691E3
:100E6400F201EE5FFF4F3F4F3BBFA791B691F201F6
:100E7400362DEC5FFF4F3F4F3BBF47915791669133
:100E8400242F252B262B21F0FA01362FD2DF01C087
:100E9400CCDF07E0400E00E0501E601EA201662D6C
:100EA4004C3B5E406140B8F20895CB081C21000021
:100EB40000A9007220BC0E01030000000001002CF8
:100EC4008131810008000037813B8103000000501C
:100ED40081000004000000568100000000000000B2
:100EE40000000075207D209520952085208D20957B
:100EF4002095209520952095209520952095209546
:100F040020952095200009021200010100C0320939
:100F140004000000FF000000120100020000004075
:100F2400EB03DD2F030000020001000300000000BA
:100F340000000000000000000000000000000000AD
:100F4400000000000000000000000000444655209E
:100F54004154584D45474136344134550004030942
:010F64000488
:0400000310000000E9
:00000001FF
